:1000000008308A00692800000A108A100A11820745
:100010004C3431343A34433453343334333431345C
:100020003034203420342034203420342034203420
:100030002034203420340D340A3400340A108A105D
:100040000A1182074C3432343A3420345634653441
:1000500072342E34203431342E3430342034203471
:10006000203420342034203420340D340A34003439
:100070000A108A100A1182074C3431343A342A3477
:100080004C3445344634543420342034253433340D
:100090002E343134663420346434423420340D3408
:1000A0000A3400340A108A100A1182074C343234A0
:1000B0003A342A345234493447344834543420349E
:1000C000253433342E3431346634203464344234AD
:1000D00020340D340A3400340A108A100A118207C1
:1000E0004C3432343A34203452344934473448346E
:1000F00054342034253433342E34313466342034AF
:100100006434423420340D340A3400340A108A1026
:100110000A1182074C3431343A3420344C3445349B
:100120004634543420342034253433342E3431349E
:10013000663420346434423420340D340A340034BC
:100140000A108A100A1182074C3431343A342A34A6
:10015000203420344D345534543445342034203444
:1001600020342034203420342034203420340D3402
:100170000A3400340A108A100A1182074C343234CF
:100180003A342A34203420344D34553454344534F0
:1001900020342034203420342034203420342034BF
:1001A00020340D340A34003433080139B4003308E4
:1001B0000239B5000310B50C33080439B600B60C8B
:1001C000B60C3F30B60533080839B700B70CB70C8A
:1001D000B70C1F30B70533081039B800B80E0F3010
:1001E000B80533082039B900B90EB90C0730B90584
:1001F00033084039BA00BA0EBA0CBA0C0330BA054B
:1002000033088039BB003B0DBB0103183B14BB080E
:10021000031D0C2906110D29061583160611061259
:1002200083120616BA08031D172906111829061588
:10023000831606110612831206120230F700F70B1E
:100240001F2900008316061283120616B908031D23
:100250002B2906112C290615831606110612831266
:1002600006120230F700F70B33290000831606123E
:1002700083120616B808031D3F29061140290615EA
:10028000831606110612831206120230F700F70BCE
:10029000472900008316061283120616B708031DAD
:1002A00053290611542906158316061106128312C6
:1002B00006120230F700F70B5B29000083160612C6
:1002C00083120616B608031D67290611682906154C
:1002D000831606110612831206120230F700F70B7E
:1002E0006F2900008316061283120616B508031D37
:1002F0007B2906117C290615831606110612831226
:1003000006120230F700F70B83290000831606124D
:1003100083120616B408031D8F29061190290615AD
:10032000831606110612831206120230F700F70B2D
:100330009729000083160612831206160230F70072
:10034000F70BA029000083160612831206128316EB
:100350000611831206110034343084008313000820
:100360000319BF290230F800F701F70BB529F80B84
:10037000B4299730F700F70BBB29800BB229003462
:1003800083168612831286120830F800C7290000EF
:10039000F817D829F813C10C03188616031C861207
:1003A0007817D8297813F80BCB29D62900008616A0
:1003B0001C308400840BDA29DD29F81BCA29781B3C
:1003C000D22900348E30F7003408F8003308F900E1
:1003D000FA01F808031DF6297908F800F901083038
:1003E000F702F808031DF629F701FE290310F81B90
:1003F000FD29F90DF80DF703F629F813003441082B
:1004000003196F2AC900450803196F2AC907031881
:10041000102A7F30C902031C6F2A03196F2A142A7D
:100420008130C90703186F2A4908F700F801F9015C
:10043000FA014208CD00CD174308CC004408CB0098
:100440001830C900CA014B1C3D2A4808FA07031C92
:100450002F2AF90A031D2F2AF80A0319CA17470879
:10046000F907031C362AF80A0319CA174608C300FD
:10047000C3174308F8070318CA17CA0DF80CF90C7C
:10048000FA0CCD0CCC0CCB0C0310C90B222A01307A
:10049000F70703186F2AF81B542ACD0DFA0DF90D32
:1004A000F80DF70303196F2ACD1F652AFA0A031DF9
:1004B000652AF90A031D652AF80A031D652AF80C46
:1004C000F90CFA0CF70A03196F2A4208CA00460809
:1004D000CA06CA1F6D2AF817732AF813732AF70180
:1004E000F801F901FA01003480308318B806BD0123
:1004F000BE013408BC003808BC0633080319642B5D
:10050000BB00F700370803196D2BBB020319092B39
:10051000031CC72A3808C100C1173908C0003A08AF
:10052000BF00BE010310C10CC00CBF0CBE0CBB0B46
:10053000912ABC1F9E2A3D14812B3D103B103D1675
:10054000363084008313962B3D12BC1BB12A3B1C12
:10055000BC2AC10CC00CBF0CBE0CF70A03197C2BC3
:10056000BC2AC11BBF2A0310BE0DBF0DC00DC10D9B
:10057000F70303197C2BB12A3D17292B3D133408AF
:10058000BC00BC1FC52AC117752BC113752B3708BA
:10059000BB00F7003308BB023408C100C11735089F
:1005A000C0003608BF00BE010310C10CC00CBF0C58
:1005B000BE0CBB0BD32ABC1FE02ABD14812BBD107F
:1005C0003B10BD163A3084008313962BBD12BC1B22
:1005D000F32A3B1CFE2AC10CC00CBF0CBE0CF70A50
:1005E00003197C2BFE2AC11B012B0310BE0DBF0D6E
:1005F000C00DC10DF70303197C2BF32ABD17292B5E
:10060000BD133808BC00BC1F072BC117752BC113C5
:10061000752B3808C100C1173908C0003A08BF005F
:10062000BC1F162BC1133D15812B3D11BE013B1084
:10063000363084008313962BBC1B3F2B3408BC0040
:100640003B1C292BC10CC00CBF0CBE0CF70A0319B4
:100650007C2BBE1F3A2BBF0A031D3A2BC00A031D79
:100660003A2BC10A031D3A2BC10CC00CBF0CF70A70
:1006700003197C2B3D1BBE2ABD1B002B5E2B80303B
:10068000C106C11F472B812B3808BC00542B3408EE
:10069000BC00C108031D542BC008031D542BBF0808
:1006A000031D542BF701752BC11B5E2B0310BE0DD0
:1006B000BF0DC00DC10DF70B542B7C2BBC1F622B43
:1006C000C117752BC113752B3708F7003808C10007
:1006D0003908C0003A08BF00752B3308F70034080A
:1006E000C1003508C0003608BF004108F8004008C6
:1006F000F9003F08FA00B42BF701F801F901FA01FB
:10070000B42BBE01BF09C009C109BE09BE0A031D41
:100710008F2BBF0A031D8F2BC00A0319C10A3D1876
:100720009D2ABD18DF2A3D19152B442B0008BF0751
:10073000031CA02BC00A031DA02BC10A03193B14E4
:1007400084030008C007031CA82BC10A03193B142B
:1007500084030008801F803AC10703183B143D1A28
:10076000A42ABD1AE62A1C2B0034F701F801F9016E
:10077000FA01C901CA01CB01CC014808470446046B
:1007800045040319F32B2030CD000310C10DC20D19
:10079000C30DC40DC90DCA0DCB0DCC0D48084C02BC
:1007A000031DDC2B47084B02031DDC2B46084A02C5
:1007B000031DDC2B45084902031CED2B4508C9022B
:1007C0004608031C460FCA024708031C470FCB020A
:1007D0004808031C480FCC020314F70DF80DF90D5F
:1007E000FA0DCD0BC52B4930840083130034040867
:1007F000B9003808BB000319162C3708C4003608A6
:10080000C3003508C2003408C100C801C701203048
:10081000C6008230C500FF217A08B7007908B6000B
:100820007808B5007708B400BB0BFD2B3708C4006F
:100830003608C3003508C2003408C1004108B63C80
:10084000C100FA014208C500C2170310C20CC30C54
:10085000C40CFA0CF90CF80CF70CC10B252CC51FB5
:100860003C2CF709F809F909FA09F70A0319F80AFB
:100870000319F90A0319FA0A7A08B7007908B600C9
:100880007808B5007708B400B71F532CB903B91620
:10089000B409B509B609B709B40A0319B50A0319A9
:1008A000B60A0319B70A3B30C0009A30BF00CA30FD
:1008B000BE00BD010A30BB0038080319B90A370869
:1008C000C4003608C3003508C2003408C10040081F
:1008D000C8003F08C7003E08C6003D08C500B52354
:1008E0000008B400840A0008B500840A0008B600B5
:1008F000840A0008B700FD308407F708031D932C15
:10090000380A3B020319932C39080319952C0F3927
:100910003B0203198D2C0318C52CB91BC52C391BA0
:10092000952C2030C12C2030B905B91EA32CB9124A
:100930003808031DB9037708B9002D30C100C02164
:100940003908F700B90138083B02031DB12C7708BC
:10095000B9002E30C100C0213908F7002030B90598
:1009600000303030B91EC12CB9123808031DB9034C
:100970007708B9002D30C100C0213908F700B9014E
:100980003030F7077708C100C0214008C4003F0895
:10099000C3003E08C2003D08C100C801C701C6012E
:1009A0000A30C500B5237A08C0007908BF0078086E
:1009B000BE007708BD00BB0B5F2C00342A08FF3C4B
:1009C000B401B300E221C401C301C2017E30C10001
:1009D0007A08C8007908C7007808C6007708C500FB
:1009E000FF218314B601B5017C30B4008330B3001D
:1009F0007A08BA007908B9007808B8007708B70013
:100A000074227A08A5007908A4007808A300770862
:100A1000A2002B08FF3CB401B300E221C401C301D2
:100A2000C2017E30C1007A08C8007908C700780882
:100A3000C6007708C500FF218314B601B5017C30DC
:100A4000B4008330B3007A08BA007908B900780896
:100A5000B8007708B70074227A08A9007908A800BE
:100A60007808A7007708A6002008013A03193F2D4F
:100A7000033A03198B2D013A0319D72D232EB30105
:100A800033083820B30AF700C100C0210A3033020E
:100A9000031D402D023084002508B7002408B6004D
:100AA0002308B5002208B4000130B800F7230F3046
:100AB000B40034083820B40AF700C100C021153052
:100AC0003402031D592D0830B400AC21B3013308A2
:100AD0005220B30AF700C100C0210A303302031DBF
:100AE000672D023084002908B7002808B6002708BF
:100AF000B5002608B4000130B800F7230F30B40069
:100B000034085220B40AF700C100C0211530340265
:100B1000031D802D232EB30133083820B30AF700BC
:100B2000C100C0210A303302031D8C2D0230840025
:100B30002508B7002408B6002308B5002208B40031
:100B40000130B800F7230F30B40034083820B40A5D
:100B5000F700C100C02115303402031DA52D083057
:100B6000B400AC21B30133086C20B30AF700C10014
:100B7000C0210A303302031DB32D0230840029083E
:100B8000B7002808B6002708B5002608B4000130D1
:100B9000B800F7230F30B40034086C20B40AF70013
:100BA000C100C02115303402031DCC2D232EB3010A
:100BB00033088620B30AF700C100C0210A3033028F
:100BC000031DD82D023084002508B7002408B60084
:100BD0002308B5002208B4000130B800F7230F3015
:100BE000B40034088620B40AF700C100C0211530D3
:100BF0003402031DF12D0830B400AC21B3013308D9
:100C00005220B30AF700C100C0210A303302031D8D
:100C1000FF2D023084002908B7002808B6002708F5
:100C2000B5002608B4000130B800F7230F30B40037
:100C300034085220B40AF700C100C0211530340234
:100C4000031D182E232E0034831605148312051855
:100C5000242EAE018316051483120518362E063095
:100C6000F700F70B312E0000AE0A2A2E2E08503C5A
:100C700003183B2EAF0A83160514831205183B2E6A
:100C8000AE0183160514831205184D2E0630F700A9
:100C9000F70B482E0000AE0A412E2E08503C0318D8
:100CA000532E0230AF078316051483120518532EF6
:100CB000AE018316051483120518652E0630F70061
:100CC000F70B602E0000AE0A592E2E08503C031878
:100CD0006B2E0430AF0783160514831205186B2E94
:100CE000AE0183160514831205187D2E0630F70019
:100CF000F70B782E0000AE0A712E2E08503C031818
:100D0000832E0830AF078316051483120518832E2F
:100D1000AE018316051483120518952E0630F700D0
:100D2000F70B902E0000AE0A892E2E08503C0318B7
:100D30009B2E1030AF0783160514831205189B2EC7
:100D4000AE018316051483120518AD2E0630F70088
:100D5000F70BA82E0000AE0AA12E2E08503C031857
:100D6000B32E2030AF078316051483120518B32E57
:100D7000AE018316051483120518C52E0630F70040
:100D8000F70BC02E0000AE0AB92E2E08503C0318F7
:100D9000CB2E4030AF078316051483120518CB2ED7
:100DA0000730B400AC210230B300F830B400083092
:100DB000B402031CE72E3430840083130310800C2C
:100DC00000080319E72EE52E0000800BE42EB30B7C
:100DD000D52E30082F02031DEF2EB20AF22E2F0857
:100DE000B000B2018A157229A1012008013A031945
:100DF000002F033A0319092F013A03190E2F132F5D
:100E00002A08C03C0318AA0A2B08C03C0318AB0AE6
:100E1000132F2A08C03C0318AA0A132F2B08C03C22
:100E20000318AB0A132FDE2403178D0103132A08BE
:100E300003178C0083168C130C15831203130B08F5
:100E4000F7008B138316031755308D00AA308D00E1
:100E50008C148C18292F0C117708831203138B0420
:100E6000013003178D0003132B0803178C00831622
:100E70008C130C15831203130B08F7008B138316C6
:100E8000031755308D00AA308D008C148C18462F16
:100E90000C117708831203138B04831686118312B7
:100EA00086112B08B300D4202A08B300D42083165F
:100EB0008611831286158A157E29A1012008013A20
:100EC0000319692F033A0319722F013A0319772F77
:100ED0007C2F2A08013C031CAA032B08013C031C9D
:100EE000AB037C2F2A08013C031CAA037C2F2B0890
:100EF000013C031CAB037C2FDE2403178D0103137D
:100F00002A0803178C0083168C130C158312031305
:100F10000B08F7008B138316031755308D00AA308A
:100F20008D008C148C18922F0C11770883120313E8
:100F30008B04013003178D0003132B0803178C005B
:100F400083168C130C15831203130B08F7008B13F5
:100F50008316031755308D00AA308D008C148C1821
:100F6000AF2F0C117708831203138B04831686119D
:100F7000831286112B08B300D4202A08B300D42092
:100F800083168611831286158A158529A101A00A68
:100F90002008033C0318CE2F0130A000DE24831666
:100FA0008611831286112B08B300D4202A08B300BF
:0E0FB000D42083168611831286158A158C298B
:10100000A108031D39288316861183128611B301A6
:101010008A11D4208A15B3018A11D4208A15831627
:10102000861183128615B30133088A11A0208A1510
:10103000B30AF700C1008A11C0218A1515303302A6
:10104000031D14280830B4008A11AC218A15B3019D
:1010500033088A11BA208A15B30AF700C1008A1131
:10106000C0218A1515303302031D28280130A10044
:10107000622803178D0183168C130C1483120C083D
:101080000313AA00013003178D0083168C130C1470
:1010900083120C080313AB0083168611831286118A
:1010A0002B08B3008A11D4208A152A08B3008A11AC
:1010B000D4208A1583168611831286158A11DE24A0
:1010C0008A15A1016430B4008A11AC218A158A15F1
:1010D0009229840183131F308305723083168F0099
:1010E0000F0886128312861683161F129F121B0882
:1010F00080399B0007309C008312A001A101A2014E
:10110000A301A401A501A601A701A801A901AA01A3
:10111000AB01AC01AD01AE01AF01B001B101B20153
:10112000703083168F000F0883121F100130831652
:10113000850000308600861183128611B3018A1162
:10114000D4208A15B3018A11D4208A1583168611FA
:10115000831286150130B4008A11AC218A158316DA
:10116000861183128611B3018A11D4208A15B30126
:101170008A11D4208A1583168611831286150A30A7
:10118000B300FA30B4008A11AC218A15B30BC12820
:10119000B30133088A1104208A15B30AF700C1008D
:1011A0008A11C0218A1515303302031DC928083061
:1011B000B4008A11AC218A15B30133088A111E20AC
:1011C0008A15B30AF700C1008A11C0218A151530AB
:1011D0003302031DDD2803178D0183168C130C14B5
:1011E00083120C080313AA00013003178D00831625
:1011F0008C130C1483120C080313AB002A08FA3C5E
:10120000031838290130AA00AB0003178D018C00A8
:1012100083168C130C15831203130B08F7008B1322
:101220008316031755308D00AA308D008C148C184E
:1012300017290C117708831203138B04013003174D
:101240008D008C0083168C130C15831203130B086E
:10125000F7008B138316031755308D00AA308D00CD
:101260008C148C1831290C117708831203138B040A
:101270000130A00083168611831286112B08B3005B
:101280008A11D4208A152A08B3008A11D4208A151D
:1012900083168611831286150830B300FA30B40025
:1012A0008A11AC218A15B30B4E298A11DE248A15C6
:1012B000AE01AF01B10183160514831205185B2935
:1012C00083160514831205186C294230F700F70BBA
:1012D00067290000B10A60293108163C03189329D8
:1012E0008A11242E8A153208023C031D9229B2016C
:1012F0002F08123C031D7F298A11F42E8A152F080E
:10130000133C031D86298A115D2F8A152F08253C61
:10131000031D8D298A11C62F8A152F08143C031D21
:10132000922900289929B2011330B4008A11AC2106
:061330008A155829630034
:04400E00703FFF3FC1
:00000001FF
